:100000000C942A001895000018950000189500001F
:10001000189500001895000018950000189500002C
:10002000189500000C94D90618950000189500004A
:10003000189500001895000018950000189500000C
:1000400018950000189500001895000018950000FC
:10005000189500008FE58DBFC4E0E0E84E2E88E0E3
:100060008EBFD8E0F7E05F2EEEEFF7E0A0E6B0E05D
:1000700088278D933197E9F7662481E48ABB81E371
:100080008BBB8FEB87BB8FEB88BB88E084BB83E0A7
:1000900085BB80E081BB8BE382BB80E08FBD81E0CC
:1000A0008EBD8FE181BD87E181BD86E086B980E4A8
:1000B00087B9C398C29AD89ADE9AC498C798C59847
:1000C000F894A8950E9406088091D30080688093D8
:1000D000D300EFEFF1E0A4ECB0E091E00E946727DD
:1000E0000091C400003081E009F080E08F9300911E
:1000F000C4000E3F80E010F009F081E09F91892B51
:10010000882311F40C9487008EEB8093C400009137
:10011000C4004AE0040F01BF89E190E00E942A2652
:10012000EAE0F0E0BB27A0E10E946427013311F46C
:100130000C94E200EAE0F0E0A0E1BB2781E38C93BD
:100140007BE70E945327EBE0F0E0A0E1BB278FE0C4
:100150008C937BE70E945327ECE0F0E001E010E095
:10016000A0E1BB277BE70E945527EEE0F0E0A0E18D
:10017000BB2780E08C937BE70E945327E2E1F0E00D
:1001800000E010E0A0E1BB277BE70E945527EFE0ED
:10019000F0E0A0E1BB2780E08C937BE70E9453272F
:1001A000E0E1F0E0A0E1BB2780E08C937BE70E94D8
:1001B0005327E1E1F0E0A0E1BB2780E08C937BE7EF
:1001C0000E945327EBE0F0E0AFEBB0E00E94642721
:1001D0000091BF00043618F011F00C94F1000C945B
:1001E000F40084E68093BF0080E797E9A0ECB0E0DC
:1001F0008D939C93ECE0F0E0AAEBB0E00E946627C0
:10020000EEE0F0E0A5ECB0E00E946427EFE0F0E063
:10021000A6ECB0E00E9464270E940A08E0E1F0E04A
:10022000AFE6B0E00E946427E1E1F0E0A0E7B0E0D3
:100230000E946427E2E1F0E0A3E6B0E00E946627B6
:10024000A3E6B0E00E942B25E2E1F0E0A3E6B0E0F7
:100250007BE70E945527AAEBB0E00D911C9100307E
:1002600050E0150711F00C943B0181E090E0AAEBFF
:10027000B0E08D939C9380E08093D20080916C00DD
:10028000877F80936C0080E08093C80086E0809335
:10029000C2008DE08093C300EBE6F0E0FA93EA93AE
:1002A0000E94A816229684E190E00E942A26DE98F9
:1002B0000E941626C49A88EC90E00E942A26A895EF
:1002C00081B5886181BD877F81BDE0E6F0E0FA936A
:1002D000EA930E94891B2296A89500916000003045
:1002E00011F40C9479010E94D11A0E94CD070C944C
:1002F0007E0180916C008E7F80936C000E94FA1AC0
:1003000084E690E00E942A2600916B00003018F0ED
:1003100011F00C948D010C949401EBE6F0E0FA934B
:10032000EA930E94E01822960027ACE6B0E08C9198
:1003300080FB0EF401E040E0041711F00C94A201E0
:100340000E940B0E82E390E00E942A267894A895E2
:1003500081B5886081BD00916F00003011F00C9470
:10036000B70181E090E0AAEBB0E08D939C930091FF
:100370006F00013011F00C94C901AAEBB0E00D91AF
:100380001C9141E050E0040F151FAAEBB0E00D9363
:100390001C93A6EBB0E04D915C91AAEBB0E00D91FF
:1003A0001C910417150718F011F00C94D9010C9446
:1003B000DF0181E090E0AAEBB0E08D939C930027F1
:1003C000ACE6B0E08C9184FB0EF401E041E0041750
:1003D00081E009F080E08F930027ACE6B0E08C91DB
:1003E00080FB0EF401E040E0041781E009F080E0BA
:1003F0009F918923882311F40C941102EAEBF0E019
:10040000FA93EA935A924A9280E0A42DB52D8C93E8
:1004100081E00E9418250E94040C249681E00E942D
:10042000142580E08093BC0080E080936B00809175
:100430006C008F7780936C000027ACE6B0E08C9165
:1004400080FB0EF401E041E0041711F00C942A0245
:100450000E940608A895ADE6B0E088278C9300912D
:10046000D200003011F00C941B03E0E6F0E0FA93A8
:10047000EA930E940017229600916000003018F065
:1004800011F00C9445020C941B0380916C00806861
:1004900080936C000091D400003011F00C9496020F
:1004A000809160008093C8000027ACE6B0E08C919A
:1004B00084FB0EF401E040E0041711F00C9470028C
:1004C000A0E6B0E08C91AAEBB0E08D9388278C93E6
:1004D000ADE6B0E0E4E2FFE40E946C260C949602E4
:1004E0000027ACE6B0E08C9181FB0EF401E041E026
:1004F000041711F00C949002A0E6B0E00D911127C2
:1005000041E050E0040F151FAAEBB0E00D931C93DF
:10051000ADE6B0E0E4E2FFE40E946C260C949602A3
:10052000ADE6B0E0E6E2FFE40E946C260091D40064
:10053000023011F00C941B03809160008093C8007E
:1005400000916000013011F00C94B20281E090E063
:10055000AAEBB0E08D939C93ADE6B0E0E4E2FFE45B
:100560000E946C2600916000023011F00C9403038D
:10057000A6EBB0E00D911C91013050E0150718F08A
:1005800011F00C94C5020C94FD02A6EBB0E00D91A5
:100590001C9141E050E0041B150BA3E6B0E00D9365
:1005A0001C9301E010E00F931F93A3E6B0E08D9140
:1005B0009C918A939A930E9446252296402F512F10
:1005C0001F910F91040F151FA5E6B0E00D931C932A
:1005D000AAEBB0E04D915C91A5E6B0E00D911C91C5
:1005E0000417150711F40C94D102A5E6B0E08D9123
:1005F0009C91AAEBB0E08D939C93ADE6B0E0E4E271
:10060000FFE40E946C2600916000033011F00C940E
:100610000F03ADE6B0E0E6E2FFE40E946C26009135
:100620006000043011F00C941B03ADE6B0E0E8E28A
:10063000FFE40E946C260027ACE6B0E08C9184FBBE
:100640000EF401E041E0041781E009F080E08F93AF
:100650000027ACE6B0E08C9181FB0EF401E041E0B4
:10066000041781E009F080E09F9189238F93009126
:10067000D200013081E009F080E09F918923882336
:1006800011F40C948603AAEBB0E00D911C9101309B
:1006900050E0150711F00C948603E0E6F0E0FA93C1
:1006A000EA930E940017229600916000003080E0DB
:1006B00010F009F081E08F93A6EBB0E04D915C91D2
:1006C000A0E6B0E00D9111270417150781E008F0AE
:1006D00080E09F918923882311F40C948603A0E67F
:1006E000B0E00D91112741E050E0040F151FAAEB77
:1006F000B0E00D931C93ADE6B0E0E4E2FFE40E94AD
:100700006C2680916C00806880936C000027ACE6BA
:10071000B0E08C9184FB0EF401E040E0041781E02E
:1007200009F080E08F930091D200013081E009F060
:1007300080E09F918923882311F40C94B703E0E6AD
:10074000F0E0FA93EA930E9400172296009160006D
:10075000003011F00C94B703ADE6B0E0EAE2FFE43C
:100760000E946C2680916C00806880936C00EBE6A0
:10077000F0E0FA93EA930E94A816229600916B008B
:10078000043011F00C94CB030E94BE0780916C00E2
:10079000806880936C0000916B00013011F00C9424
:1007A000DC03ADE6B0E0E6E2FFE40E946C26809157
:1007B0006C00806880936C0080E080936000009102
:1007C0006B00023081E009F080E08F930091BF0060
:1007D000043681E008F080E09F918923882311F49A
:1007E0000C94FA03AFEBB0E08C918B5F8C9381E0BB
:1007F0008093600000916B00033081E009F080E09D
:100800008F930091BF00053081E009F080E09F9157
:100810008923882311F40C94130481E08093BF0092
:1008200081E08093600000916B00033081E009F06B
:1008300080E08F930091BF00053080E010F009F058
:1008400081E09F918923882311F40C942F04AFEB4E
:10085000B0E08C9185508C9381E080936000009192
:100860006000013011F00C945C048EB5887F8EBD61
:100870005A924A928091BF00A42DB52D8C9381E0AD
:100880000E9418250E949621229681E00E9414253C
:10089000EBE0F0E0AFEBB0E07BE70E945327009184
:1008A000D200013011F00C94570481E08EBD80918C
:1008B0006C00806880936C00EDE6F0E0ADE6B0E09F
:1008C0000E947626ADE6B0E08C91803081E009F49C
:1008D00080E08F9300916B00003081E009F480E0AC
:1008E0009F91892B8F930091BC00013081E009F02A
:1008F00080E09F91892B882311F40C941C020091B5
:10090000BC00013011F00C94A60480E08093BC0080
:10091000ADE6B0E0E6E2FFE40E946C260027ACE61C
:10092000B0E08C9181FB0EF401E041E0041711F07E
:100930000C94A60481E090E0AAEBB0E08D939C9328
:10094000ADE6B0E0E4E2FFE40E946C26ADE6B0E084
:10095000E4E2FFE40E947E2711F00C941805009158
:10096000D200013011F00C94B7040E94BE07A6EB30
:10097000B0E04D915C91AAEBB0E00D911C91041791
:10098000150718F011F00C9413050027ACE6B0E041
:100990008C9180FB0EF401E040E0041711F00C9400
:1009A000E404EAEBF0E0FA93EA935A924A9280E088
:1009B000A42DB52D8C9381E00E9418250E94040C73
:1009C000249681E00E9414250027ACE6B0E08C91CB
:1009D00080FB0EF401E041E0041711F00C941105C6
:1009E0000E94CD070027ACE6B0E08C9180FB0EF4AE
:1009F00001E040E0041711F00C941105EAEBF0E07F
:100A0000FA93EA935A924A9280E0A42DB52D8C93E2
:100A100081E00E9418250E94040C249681E00E9427
:100A200014250C94160580E08093C8000C944606AB
:100A3000E6E2FFE40E947E2711F00C94B0050091DD
:100A4000D200013011F00C9427050E94BE07AAEBDA
:100A5000B0E00E942B250027A3EDB0E08C9187FB2E
:100A60000EF401E041E0041711F00C944C0500274E
:100A7000ACE6B0E08C9184FB0EF401E040E004179A
:100A800011F00C944705AAEBB0E00E94322580914A
:100A9000D3008F778093D300A6EBB0E04D915C91AB
:100AA000AAEBB0E00D911C910417150718F011F096
:100AB0000C945C050C94620581E090E0AAEBB0E038
:100AC0008D939C930027ACE6B0E08C9180FB0EF4F4
:100AD00001E040E0041711F00C948105EAEBF0E02E
:100AE000FA93EA935A924A9280E0A42DB52D8C9302
:100AF00081E00E9418250E94040C249681E00E9447
:100B000014250027ACE6B0E08C9180FB0EF401E0E8
:100B100041E0041711F00C94AE050E94CD070027A8
:100B2000ACE6B0E08C9180FB0EF401E040E00417ED
:100B300011F00C94AE05EAEBF0E0FA93EA935A92C6
:100B40004A9280E0A42DB52D8C9381E00E94182557
:100B50000E94040C249681E00E9414250C94460601
:100B6000E8E2FFE40E947E2711F00C942806009131
:100B7000D200013011F00C94BF050E94BE07AAEB11
:100B8000B0E00D911C91013050E0150718F011F004
:100B90000C94CC050C94D205AAEBB0E00E9432254F
:100BA0000C94DA05A6EBB0E08D919C91AAEBB0E035
:100BB0008D939C930027ACE6B0E08C9180FB0EF403
:100BC00001E040E0041711F00C94F905EAEBF0E0C5
:100BD000FA93EA935A924A9280E0A42DB52D8C9311
:100BE00081E00E9418250E94040C249681E00E9456
:100BF00014250027ACE6B0E08C9180FB0EF401E0F8
:100C000041E0041711F00C9426060E94CD0700273E
:100C1000ACE6B0E08C9180FB0EF401E040E00417FC
:100C200011F00C942606EAEBF0E0FA93EA935A925C
:100C30004A9280E0A42DB52D8C9381E00E94182566
:100C40000E94040C249681E00E9414250C94460610
:100C5000EAE2FFE40E947E2711F00C9436060E941F
:100C6000BE0780E08093C8000C944606ECE2FFE4E7
:100C70000E947E2711F00C944606ECE0F0E0AAEB0F
:100C8000B0E07BE70E9455270C94460681E090E097
:100C90000E942A260027ACE6B0E08C9187FB0EF478
:100CA00001E040E0041718F011F00C9459060C9480
:100CB000D70600916B00003018F011F00C9462061A
:100CC0000C94C906A895E0E6F0E0FA93EA930E9436
:100CD000A816229600916000043011F00C94BD0615
:100CE0000E94BE0780E08093C8000E94080885E04B
:100CF00090E00E942A2680E080936200E0E6F0E027
:100D0000FA93EA930E94A8162296A2E6B0E08C918C
:100D10008F5F8C9388E090E00E942A26009160000B
:100D2000003081E009F080E08F930091620004368A
:100D300080E010F009F081E09F91892B882311F465
:100D40000C947E0600916200043618F011F00C94A9
:100D5000AB060C94BA0681B5886181BD877F81BDE1
:100D6000E3E6F0E0FA93EA930E947C08229681B5CC
:100D7000886081BD80E08093600081E090E00E9407
:100D80002A2600916000003011F00C9462060C9449
:100D9000CD068AE090E00E942A260091D200003021
:100DA00011F00C94D70685E090E00E942A260C945E
:100DB00017020F921F922F923F924F925F927F9253
:100DC000AF92BF920F931F932F933F934F935F93D5
:100DD0006F937F938F939F93AF93BF93CF93DF9343
:100DE000EF93FF938FB78F93F89489B78B7F89BF69
:100DF0008EB5887F8EBD5A924A9280E092E0A42DF3
:100E0000B52D8D939C9382E00E9418250E94922418
:100E1000229682E00E9414250091DD000A3011F034
:100E20000C9414070E9406080E94161E0091DD0013
:100E30000A3011F00C9421070E94080880E080938A
:100E4000DD00ADEDB0E08C918F5F8C93A89500270D
:100E5000ACE6B0E08C9180FB0EF401E040E00417BA
:100E600011F00C9446075A924A9280E092E0A42D29
:100E7000B52D8D939C9382E00E9418250E949224A8
:100E8000229682E00E9414250E94161EA9EDB0E071
:100E90004D915D916D917C91A5EDB0E00D911D910D
:100EA0002D913C910E94CA2680E00CF481E08F9342
:100EB0000027ACE6B0E08C9180FB0EF401E040E04E
:100EC000041781E009F080E09F918923882311F4C1
:100ED0000C94770780E49CE990934D0080934C003C
:100EE00081E08EBD89B7846089BF0C94A00780E043
:100EF0008093D20080916C00877F80936C000027E4
:100F0000ACE6B0E08C9180FB0EF401E040E0041709
:100F100011F00C949407ACE6B0E08C9184FBACEB40
:100F2000B0E0882780F98C930091C5004FE7042337
:100F3000A1E6B0E00C930E94080880E08093C8000E
:100F40008F918FBFFF91EF91DF91CF91BF91AF91C3
:100F50009F918F917F916F915F914F913F912F91D1
:100F60001F910F91BF90AF907F905F904F903F90F7
:100F70002F901F900F901895F894FFCF89B78B7F13
:100F800089BF8EB5887F8EBD80E08093D20080912E
:100F90006C00877F80936C000895DE9A6E98C498E9
:100FA000C598C7980E940808E2E0F0E00E94A125D9
:100FB000DE98C49A0E94162684E690E00E942A26B3
:100FC000A89580916C008E7F80936C00E0E6F0E045
:100FD000FA93EA930E94891B2296009160000030E8
:100FE00011F40C94030880916C00816080936C0074
:100FF00084E690E00E942A26DE9A6E98C498C598EE
:10100000C7980C9405080E940B0E0895AB9808959C
:10101000AB9A089581E00E94392680916C008F7E02
:1010200080936C000091C50041E00423A881B98140
:101030000C93A881B9810C91003011F40C9425080F
:1010400080916C00806180936C0080916C008D7F3A
:1010500080936C000091C50042E00423A881B9810F
:101060000C93A881B9810C91003011F40C943D08C7
:1010700080916C00826080936C0080916C008F7D09
:1010800080936C000091C50040E20423A881B981DF
:101090000C93A881B9810C91003011F40C9455087F
:1010A00080916C00806280936C008091D3008F7B74
:1010B0008093D3000091C60046E00423A881B98143
:1010C0000C93A881B9810C9142E00E946E270C9389
:1010D000A881B9818C918093D4000091D400033011
:1010E00011F00C94760882E08093D40081E0481AD5
:1010F0008827580A2296089582E00E94392681E0C6
:101100000E94392681E00E94392680E0AA81BB81B5
:101110008C9383E4A0EAB0E08C938FE4A1EAB0E082
:101120008C938EE4A2EAB0E08C9386E4A3EAB0E06C
:101130008C9389E4A4EAB0E08C93ACE6B0E08C91A7
:1011400085FBA881B981882780F98C9380916C00F8
:10115000806280936C00A6E7B0E00D911D912D9107
:101160003C91A6E9B0E00D931D932D933C935A92C8
:101170004A92A6E9B0E00D911D912D913C91A42DCC
:10118000B52D0D931D932D933C9384E00E9418255B
:101190005A924A9280E090E0A42DB52D8D939C93B5
:1011A00082E00E9418255A924A9281E0A42DB52D22
:1011B0008C9381E00E9418250E941A0F269687E0E2
:1011C0000E9414258FE00E943926E8EAF0E006E04C
:1011D000A881B9810E944527A881B981EEE2FFE488
:1011E0000E947E270FB68FE0481A8827580A229659
:1011F0000FBE81E009F080E08F93009191000031F3
:1012000081E009F080E09F918923882311F40C94F8
:10121000570981E0AA81BB818C93A6E9B0E00D91CA
:101220001D912D913C91A6E7B0E00D931D932D9358
:101230003C9380916C008F7D80936C005A924A920F
:10124000A6E9B0E00D911D912D913C91A42DB52DF5
:101250000D931D932D933C9384E00E9418255A9280
:101260004A9280E090E0A42DB52D8D939C9382E06E
:101270000E9418255A924A9280E0A42DB52D8C9395
:1012800081E00E9418250E941A0F269687E00E948E
:101290001425A6E9B0E00D911D912D913C91A6E792
:1012A000B0E00D931D932D933C930E94B109A8814A
:1012B000B9818C9180FBACE6B0E08C9185F98C9380
:1012C000AAE7B0E00D911D912D913C91A6E7B0E009
:1012D0000D931D932D933C93A6E7B0E00D911D91C6
:1012E0002D913C91A6E9B0E00D931D932D933C9375
:1012F0005A924A92A6E9B0E00D911D912D913C9130
:10130000A42DB52D0D931D932D933C9384E00E9445
:1013100018255A924A9280E090E0A42DB52D8D9325
:101320009C9382E00E9418255A924A9280E0A42D54
:10133000B52D8C9381E00E9418250E941A0F2696E5
:1013400087E00E941425AA81BB818C91AE81BF8168
:101350008D9388278C9384E0481A8827580A26960C
:10136000089582E00E94392681E00E94392681E0BA
:101370000E943926789481E090E0AC81BD818D9304
:101380009C93EA81FB81FA93EA93EE81FF81FA93C1
:10139000EA930E94C70B2496AA81BB810C9101306D
:1013A00011F00C94DE0982E090E0AC81BD818D9358
:1013B0009C9381E08093C5000C94FA09023011F0EF
:1013C0000C94ED0983E090E0AC81BD818D939C93FA
:1013D00080E08093C5000C94FA09033011F00C945E
:1013E000FA0984E090E0AC81BD818D939C9383E009
:1013F0008093C500EEE0F0E0A5ECB0E07BE70E9452
:101400005327EC81FD81FA93EA935A924A9280E045
:10141000A42DB52D8C9381E00E9418250E94040C08
:10142000249681E00E9414250091D200003011F032
:101430000C94140A88EC90E00E942A2685E090E043
:10144000AC81BD818D939C93EA81FB81FA93EA93F1
:10145000EE81FF81FA93EA930E94C70B2496EEE097
:10146000F0E0A5ECB0E00E946427AA81BB810C915A
:10147000033011F00C943E0A0C94DB0AAA81BB8164
:101480000C91013011F00C944C0AA5ECB0E08C9159
:1014900088608C930C94550A023011F00C94550A14
:1014A000A5ECB0E08C91877F8C93EEE0F0E0A5ECAA
:1014B000B0E07BE70E94532788EC90E00E942A2648
:1014C00086E090E0AC81BD818D939C93EA81FB81A5
:1014D000FA93EA93EE81FF81FA93EA930E94C70B95
:1014E0002496AA81BB810C91033011F00C947A0AE6
:1014F0000C94DB0AEEE0F0E0A5ECB0E00E9464277B
:10150000AA81BB810C91013011F00C948E0AA5ECDC
:10151000B0E08C9184608C930C94970A023011F0A7
:101520000C94970AA5ECB0E08C918B7F8C93EEE045
:10153000F0E0A5ECB0E07BE70E94532788EC90E058
:101540000E942A2687E090E0AC81BD818D939C9318
:10155000EA81FB81FA93EA93EE81FF81FA93EA93A1
:101560000E94C70B2496EEE0F0E0A5ECB0E00E94EC
:101570006427AA81BB810C91013011F00C94C70A39
:10158000A5ECB0E08C9180628C930C94D00A023070
:1015900011F00C94D00AA5ECB0E08C918F7D8C9367
:1015A000EEE0F0E0A5ECB0E07BE70E94532788EC8A
:1015B00090E00E942A2688E090E0AC81BD818D9366
:1015C0009C93EC81FD81FA93EA930E94A50B2296ED
:1015D0000091C50043E00423A881B9810C93A88140
:1015E000B9810C91003011F00C94FE0A83E090E078
:1015F000AC81BD818D939C930C94140B013011F040
:101600000C940A0B82E090E0AC81BD818D939C9399
:101610000C94140B033011F00C94140B84E090E044
:10162000AC81BD818D939C93EC81FD81FA93EA930B
:101630000E94A50B22960091C50048E00423A881D2
:10164000B9810C93A881B9810C91003011F00C94F0
:10165000310B8AE090E0AC81BD818D939C930C941A
:101660003B0B083011F00C943B0B89E090E0AC810F
:10167000BD818D939C93EC81FD81FA93EA930E9446
:10168000A50B22960091C50044E00423A881B981EE
:101690000C93A881B9810C91003011F00C94580B77
:1016A0008BE090E0AC81BD818D939C930C94620B98
:1016B000043011F00C94620B8CE090E0AC81BD81A1
:1016C0008D939C93EC81FD81FA93EA930E94A50B84
:1016D00022960091C50040E20423A881B9810C93B1
:1016E000A881B9810C91003011F00C947F0B8DE032
:1016F00090E0AC81BD818D939C930C94890B00325A
:1017000011F00C94890B8EE090E0AC81BD818D933B
:101710009C93EC81FD81FA93EA930E94A50B22969B
:101720008FE090E0AC81BD818D939C93EC81FD8135
:10173000FA93EA930E94A50B22960E940A0884E07D
:10174000481A8827580A26960895E881F981FA935D
:10175000EA935A924A9280E0A42DB52D8C9381E0B1
:101760000E9418250E94040C249681E00E941425F2
:1017700082E390E00E942A260091D200003011F00E
:101780000C94BC0B82E390E00E942A26089581E02D
:101790000E943926EA81FB81FA93EA935A924A928F
:1017A00080E0A42DB52D8C9381E00E9418250E9425
:1017B000040C249681E00E94142584E690E00E94A7
:1017C0002A26E881F981FA93EA930E94A8162296C4
:1017D000A881B9810C91003018F011F00C94F20B33
:1017E0000C94E10B0E94BE0784E190E00E942A263F
:1017F000A881B9818C91AC81BD818C9381E0481A1C
:101800008827580A2296089582E00E94392681E0AE
:101810000E9439268EB5887F8EBD80916C00877FAF
:1018200080936C00A6E7B0E00D911D912D913C9145
:10183000A6E9B0E00D931D932D933C935A924A92E2
:10184000A6E9B0E00D911D912D913C91A42DB52DEF
:101850000D931D932D933C9384E00E9418255A927A
:101860004A92AA85BB858D919C91A42DB52D8D930F
:101870009C9382E00E9418255A924A9280E0A42DFF
:10188000B52D8C9381E00E9418250E941A0F269690
:1018900087E00E94142540E050E060E070E0A2E99B
:1018A000B0E00D911D912D913C910E94CA2611F03E
:1018B0000C945C0C0C94050E0E944A215A924A9298
:1018C0008091BF00A42DB52D8C9381E00E94182536
:1018D0000E949621229681E00E9414255A924A92F3
:1018E000A0ECB0E08D919C91A42DB52D8D939C938F
:1018F00082E00E9418250E942E22229682E00E94F9
:101900001425A6E9B0E00D911D912D913C91A5ED16
:10191000B0E00D931D932D933C93A6E9B0E00D919B
:101920001D912D913C91A2E9B0E04D915D916D9199
:101930007C910E94C026A9EDB0E00D931D932D93DC
:101940003D9380E0A881B9818C930E94161E81E0AE
:1019500090E0AA81BB818D939C93AA81BB810D915C
:101960001C910F3F51E0150718F011F00C94E70C93
:10197000AA81BB81AD90BC90ADEDB0E0AA0DBB1DBE
:101980000C910F3F81E009F080E08F93AA81BB8129
:10199000AD90BC90AEEDB0E0AA0DBB1D0C910F3E1A
:1019A00080E010F009F081E09F918923882311F4F1
:1019B0000C94E00C81E0A881B9818C930C94E70C25
:1019C000AA81BB810E942B2510F40C94AD0CA88138
:1019D000B9810C91013011F00C94A50CAA81BB8146
:1019E000AD90BC90AFEDB0E0AA0DBB1D8C91AA816B
:1019F000BB818D9388278C93AA81BB810D911C910B
:101A000040E150E00E948025AA81BB814D935C9308
:101A100080E18093C700AA81BB810D911C910130A8
:101A200050E0150711F00C941A0D84E08093C70064
:101A30000C94A70D023050E0150711F00C94250D01
:101A400085E08093C7000C94A70D033050E0150784
:101A500011F00C94300D86E08093C7000C94A70D14
:101A6000043050E0150711F00C943B0D87E0809393
:101A7000C7000C94A70D053050E0150711F00C9429
:101A8000460D88E08093C7000C94A70D063050E007
:101A9000150711F00C94510D8AE08093C7000C9447
:101AA000A70D073050E0150711F00C945C0D8CE089
:101AB0008093C7000C94A70D083050E0150711F073
:101AC0000C94670D8EE08093C7000C94A70D09302D
:101AD00050E0150711F00C94720D80E18093C7005F
:101AE0000C94A70D0A3050E0150711F00C947D0DF1
:101AF00084E18093C7000C94A70D0B3050E01507CC
:101B000011F00C94880D88E18093C7000C94A70D08
:101B10000C3050E0150711F00C94930D8CE180937C
:101B2000C7000C94A70D0D3050E0150711F00C9470
:101B30009E0D80E28093C7000C94A70D0E3050E0FC
:101B4000150711F00C94A70D88E28093C700A2E955
:101B5000B0E00D911D912D913C9140E052E060E08C
:101B600070E00E944926A7E6B0E00D931D932D93E7
:101B70003D93A7E6B0E00D911D912D913C91A7EC0E
:101B8000B0E04C915527662777270E94AA25A7E643
:101B9000B0E04D935D936D937D93A7E6B0E00D911A
:101BA0001D912D913C9148EE53E060E070E00E9461
:101BB000AA25A7E6B0E04D935D936D937D93AC812C
:101BC000BD810C91003011F00C94050E00916F0056
:101BD000013011F00C94F30DECE0F0E0AAEBB0E072
:101BE0007BE70E94552781E08093D20088EC9FEA32
:101BF00090934D0080934C0089B7846089BF81E049
:101C00008EBD85E090E00E942A2683E0481A88274E
:101C1000580A24960895A895A6E7B0E00D911D9165
:101C20002D913C91AAE7B0E00D931D932D933C9329
:101C3000A6E7B0E00D911D912D913C91A6E9B0E091
:101C40000D931D932D933C935A924A92A6E9B0E0CE
:101C50000D911D912D913C91A42DB52D0D931D93AA
:101C60002D933C9384E00E9418255A924A9280E07A
:101C700090E0A42DB52D8D939C9382E00E941825B1
:101C80005A924A9280E0A42DB52D8C9381E00E9457
:101C900018250E941A0F269687E00E941425A89501
:101CA000A6EBB0E00D911C91013050E0150710F04B
:101CB0000C94810E5A924A9281E0A42DB52D8C93FA
:101CC00081E00E9418250E948822229681E00E94CD
:101CD00014258CE291E00E942A265A924A9280E0D2
:101CE000A42DB52D8C9381E00E9418250E94882296
:101CF000229681E00E94142580916C00816080937F
:101D00006C00A895A6E7B0E00D911D912D913C9136
:101D1000A6E9B0E00D931D932D933C93AAEBB0E0A0
:101D20000D911C91003050E0150781E009F080E032
:101D30008F93A6EBB0E04D915C91AAEBB0E00D91D2
:101D40001C910417150780E010F009F081E09F91C5
:101D5000892B882311F40C94B30E81E090E0AAEB58
:101D6000B0E08D939C930E940808089584E00E943F
:101D70003926A5EDB0E00D911D912D913C91A881E2
:101D8000B9810D931D932D933C93A6E7B0E00D917F
:101D90001D912D913C91A6E9B0E00D931D932D93DB
:101DA0003C935A924A92A6E9B0E00D911D912D9173
:101DB0003C91A42DB52D0D931D932D933C9384E060
:101DC0000E9418255A924A928FE19EE4A42DB52DC7
:101DD0008D939C9382E00E9418255A924A9280E04B
:101DE000A42DB52D8C9381E00E9418250E941A0F16
:101DF000269687E00E941425A6E7B0E00D911D917C
:101E00002D913C91A6E9B0E00D931D932D933C9349
:101E1000A881B9810D911D912D913C91A5EDB0E066
:101E20000D931D932D933C9384E0481A8827580AFC
:101E30002296089581E00E94392681E00E94392689
:101E400081E00E94392680E090E0A8EBB0E08D931D
:101E50009C9380916C008F7B80936C0000E010E07D
:101E600020E030E0A2E9B0E00D931D932D933C9368
:101E70000027ACE6B0E08C9185FB0EF401E041E078
:101E8000041781E009F080E08F93A885B9850D9152
:101E90001C91003050E0150781E009F480E09F912B
:101EA00089238F93AE81BF810C91003081E009F0CE
:101EB00080E09F918923882311F40C94BA0FAAE93A
:101EC000B0E0E885F9850E94DD26EAE9F0E0A8E6C1
:101ED000B7E00E943927E8E6F7E0AAE9B0E0112769
:101EE000222704E033270E94822681E4AC81BD8151
:101EF0008C93AC81BD818C918093A00081E0EAE954
:101F0000F0E001E00A93ADE6B0E00E943E27ADE6C6
:101F1000B0E08C91A1EAB0E08C9382E0EAE9F0E0D5
:101F200001E00A93ADE6B0E00E943E27ADE6B0E0E6
:101F30008C91A2EAB0E08C9383E0EAE9F0E001E062
:101F40000A93ADE6B0E00E943E27ADE6B0E08C918A
:101F5000A3EAB0E08C9384E0EAE9F0E001E00A93C0
:101F6000ADE6B0E00E943E27ADE6B0E08C91A4EA79
:101F7000B0E08C9389B78B7F89BF8EB5887F8EBD8B
:101F800081B5886181BD877F81BDAEECB0E00D91E8
:101F90001D912D913C91AAECB0E00D931D932D93D2
:101FA0003C93AAE7B0E04D915D916D917C91A6E7DD
:101FB000B0E00D911D912D913C910E94CA2611F027
:101FC0000C94EC0F02E010E020E030E0AAECB0E06E
:101FD0000D931D932D933C9380E0A881B9818C9340
:101FE000EA81FB81FA93EA935A924A92AE85BF85C1
:101FF0000D911D912D913C91A42DB52D0D931D9307
:102000002D933C9384E00E9418250E94DF1F2496A4
:1020100084E00E941425AA81BB810C910E3F11F42B
:102020000C941E1080916C00816080936C008091F4
:102030006C00806480936C000C9431105A924A9228
:10204000AA85BB858D919C91A42DB52D8D939C93D4
:1020500082E00E9418250E943411229682E00E949C
:102060001425A881B9818C918F5F8C934091730066
:10207000A881B9810C91041781E009F080E08F9369
:102080000027ACE6B0E08C9186FB0EF401E041E065
:10209000041781E009F480E09F918923882311F4DB
:1020A0000C94E710009182000B3011F00C94941006
:1020B000EAECF0E0FA93EA935A924A92AAECB0E082
:1020C0000D911D912D913C91A42DB52D0D931D9336
:1020D0002D933C9384E00E9418250E944C15249671
:1020E00084E00E941425EA85FB85FA93EA935A92CC
:1020F0004A92AAECB0E00D911D912D913C91A42D36
:10210000B52D0D931D932D933C9384E00E941825CB
:102110000E94E214249684E00E94142580E0A881A5
:10212000B9818C930C94E510AAE7B0E04D915D91D4
:102130006D917C91A6E7B0E00D911D912D913C91A0
:102140000E94CA2611F00C94AB10AA85BB850E9490
:102150001C250C94E510EAECF0E0FA93EA935A920D
:102160004A92AAECB0E00D911D912D913C91A42DC5
:10217000B52D0D931D932D933C9384E00E9418255B
:102180000E944C15249684E00E941425EA85FB8564
:10219000FA93EA935A924A92AAECB0E00D911D91FB
:1021A0002D913C91A42DB52D0D931D932D933C9312
:1021B00084E00E9418250E94E214249684E00E9484
:1021C000142580E0A881B9818C930C94EB10AA852A
:1021D000BB850E941C250027ACE6B0E08C9186FBF5
:1021E0000EF401E041E0041711F00C94F00FC49AD2
:1021F000A885B9850D911C91003050E0150711F0AC
:102200000C940A11A8EBB0E08D919C91A6EBB0E084
:102210008D939C930091D200013081E009F080E021
:102220008F930027ACE6B0E08C9180FB0EF401E0C8
:1022300040E0041781E009F080E09F918923882322
:1022400011F40C942E1180E593EC90934D00809343
:102250004C0081E08EBD89B7846089BF83E0481A55
:102260008827580A2696089584E00E94392684E03B
:102270000E94392681E00E94392681E00E94392699
:1022800081E00E94392681E00E94392680E0AE81FB
:10229000BF818C93AE81BF810C910F3018F011F08B
:1022A0000C94EF1281E0AC81BD818C93AC81BD8137
:1022B0000C910C3018F011F00C9476118FEF0E94F5
:1022C0001D260E941F260E941E26AC81BD81AD9056
:1022D000BB24A4E8B0E0AA0DBB1D8C93AC81BD81EA
:1022E0008C918F5F8C9310F40C9456118DE0AC811F
:1022F000BD818C93AC81BD810C91043118F011F03B
:102300000C9494118FEF0E941D260E941F260E949C
:102310001E26A881B9818C93AC81BD818C918F5F81
:102320008C9310F40C947A11EA85FB85FA93EA9366
:10233000EA85FB85FA93EA930E9477132496002797
:10234000ACE6B0E08C9186FB0EF401E041E00417AE
:1023500011F00C94AD110C94E71280E0AA81BB81BE
:102360008C9300919000003281E009F080E08F931F
:1023700000919000003181E009F080E09F91892B6D
:10238000882311F40C94C81181E0AA81BB818C933D
:1023900000918500003081E009F480E08F93009186
:1023A0008500053E81E009F480E09F9189238F93A9
:1023B000AA81BB810C91013081E009F080E09F91FE
:1023C0008923882311F40C94DC12009190000032D0
:1023D00011F00C94EF11A8EBB0E00E942B25002720
:1023E000ACE6B0E08C9185FB0EF401E040E0041710
:1023F00011F00C94241281E0AC81BD818C93AC85EA
:10240000BD854D915C91A8EBB0E00D911C91041736
:10241000150781E009F080E08F93A8EBB0E00D9103
:102420001C91003050E0150780E010F009F081E0C9
:102430009F918923882311F40C94221280E0AC81AF
:10244000BD818C930C94581280E0AC81BD818C933B
:1024500081E0A881B9818C93A881B9810C91053064
:1024600018F011F00C945812A881B981AD90BB24DA
:10247000AFE9B0E0AA0DBB1D4C91A881B981AD9028
:10248000BB24A4E8B0E0AA0DBB1D0C91041711F405
:102490000C94501281E0AC81BD818C930C94581245
:1024A000A881B9818C918F5F8C9310F40C942C12BD
:1024B000AC81BD810C91003081E009F080E08F9308
:1024C000AC85BD850D911C910F315EE4150781E04F
:1024D00009F080E09F91892B882311F40C94DC1281
:1024E0000E940913A885B9850D911D912D913C91EC
:1024F00040E052E060E070E00E94AA25A2E9B0E06E
:102500004D935D936D937D93E6E9F0E0FA93EA9342
:102510005A924A92AE85BF850D911D912D913C91A5
:10252000A42DB52D0D931D932D933C9384E00E9413
:1025300018250E94E214249684E00E9414258091BC
:10254000900080939100AC85BD850D911C910F3159
:102550005EE4150711F00C94AD12AC81BD810C91B5
:10256000003011F00C94DC1280916C008064809338
:102570006C0000919100003181E009F080E08F93C0
:10258000AC85BD850D911C910F315EE4150781E08E
:1025900009F480E09F918923882311F40C94DC12C4
:1025A000AA85BB850D911D912D913C91AEECB0E0BB
:1025B0000D931D932D933C9300918500003011F0F5
:1025C0000C94E71280916C00806480936C00AE8163
:1025D000BF818C918F5F8C9310F40C944A118FEF14
:1025E0000E941D260E941F260E941E26A0E6B0E023
:1025F0008C938FEF0E941D260E941F260E941E268C
:10260000A0E6B0E08C938CE0481A8827580A2C96F4
:10261000089581E00E943926A8EAB0E088278C93CB
:1026200081E0A881B9818C93A881B9810C9108308F
:1026300018F011F00C944313A881B981AD90BB241C
:10264000A4E8B0E0AA0DBB1D0C91003211F40C946B
:102650003B13A881B981AD90BB24A4E8B0E0AA0DDA
:10266000BB1D8C91A8EAB0E08F930E949A258F91B0
:102670008D9388278C93A881B9818C918F5F8C93DF
:1026800010F40C941413A8EAB0E00E949A25E6E333
:10269000FFE40E946C2689E0A881B9818C93A8810F
:1026A000B9810C910B3018F011F00C947113A881C2
:1026B000B981AD90BB24A4E8B0E0AA0DBB1D8C91FC
:1026C000A8EAB0E08F930E949A258F918D93882776
:1026D0008C93A881B9818C918F5F8C9310F40C94AA
:1026E0004F1381E0481A8827580A2296089581E0FE
:1026F0000E94392681E00E94392684E00E94392612
:102700008FEF0E941D260E941F260E941E26AC816C
:10271000BD818C938FEF0E941D260E941F260E9470
:102720001E26AA81BB818C93AA81BB810C911127A3
:102730002227332740E051E060E070E00E94492604
:10274000A885B9850D931D932D933D93A885B985D3
:102750000D911D912D913C91AC81BD814C915527DE
:10276000662777270E94C026A885B9850D931D93FB
:102770002D933D93A885B9850D911D912D913C9187
:1027800040E050E061E070E00E944926A881B981F4
:102790000D931D932D933D938FEF0E941D260E9454
:1027A0001F260E941E26AC81BD818C938FEF0E9454
:1027B0001D260E941F260E941E26AC81BD818C937F
:1027C0008FEF0E941D260E941F260E941E26AC81AC
:1027D000BD818C938FEF0E941D260E941F260E94B0
:1027E0001E26AC81BD818C938FEF0E941D260E9416
:1027F0001F260E941E26AC81BD818C938FEF0E9404
:102800001D260E941F260E941E26AA81BB818C9332
:10281000AA81BB810C9111272227332740E051E088
:1028200060E070E00E944926A885B9850D931D934C
:102830002D933D93A885B9850D911D912D913C91C6
:10284000AC81BD814C915527662777270E94C02611
:10285000A885B9850D931D932D933D93A885B985C2
:102860000D911D912D913C91A881B9814D915D9162
:102870006D917C910E94C026A885B9850D931D930A
:102880002D933D938FEF0E941D260E941F260E94CC
:102890001E26AC81BD818C938FEF0E941D260E9465
:1028A0001F260E941E26AA81BB818C93AA81BB8110
:1028B0000C9111272227332740E051E060E070E0BF
:1028C0000E944926A881B9810D931D932D933D93B4
:1028D000A881B9810D911D912D913C91AC81BD8153
:1028E0004C915527662777270E94C026A881B98179
:1028F0000D931D932D933D938FEF0E941D260E94F3
:102900001F260E941E26AC81BD818C938FEF0E94F2
:102910001D260E941F260E941E26AA81BB818C9321
:10292000AA81BB810C9111272227332740E051E077
:1029300060E070E00E944926AE81BF810D931D9337
:102940002D933D93AE81BF810D911D912D913C91B1
:10295000AC81BD814C915527662777270E94C02600
:10296000AE81BF810D931D932D933D93AE81BF81A9
:102970000D911D912D913C9140E050E061E070E09F
:102980000E944926AE81BF810D931D932D933D93E7
:10299000AE81BF810D911D912D913C91A881B9818E
:1029A0004D915D916D917C910E94C026AE81BF8159
:1029B0000D931D932D933D9386E0481A8827580A5E
:1029C0002696089584E00E94392684E00E943926E4
:1029D000AC81BD810D911D912D913C9142E050E063
:1029E00060E070E00E94C526A881B9810D931D9317
:1029F0002D933D93A3E7B0E00C91112722273327B5
:102A0000A881B9814D915D916D917C910E9449267B
:102A1000AA81BB810D931D932D933D93AA81BB8108
:102A20000D911D912D913C91AAE7B0E04D915D91E2
:102A30006D917C910E94C026AA81BB810D931D934C
:102A40002D933D93009182000B3011F40C943A15B4
:102A5000AA81BB810D911D912D913C9140E250E0E6
:102A600060E070E00E94C026AA81BB810D931D9397
:102A70002D933D93AA81BB810D911D912D913C9188
:102A8000AE81BF810D931D932D933C9388E0481A2E
:102A90008827580A2496089584E00E94392682E007
:102AA0000E943926009182000B3011F00C94901591
:102AB000AC81BD810D911D912D913C9140E850E07C
:102AC00060E070E00E94AA25A5EDB0E04D935D9313
:102AD0006D937D93AC81BD810D911C9140E850E0D8
:102AE0000E948025A881B9810D931C93A881B9818A
:102AF0000D911C9144E050E00E943F26A881B981CD
:102B00000D931C93A881B9810D911C9144E050E074
:102B1000040F151FA881B9810D931C930C94C61541
:102B2000AC81BD810D911D912D913C9140E051E012
:102B300060E070E00E94AA25A5EDB0E04D935D93A2
:102B40006D937D93AC81BD810D911C9140E051E06E
:102B50000E948025A881B9810D931C93A881B98119
:102B60000D911C9142E050E00E943F26A881B9815E
:102B70000D931C93A881B9810D911C9142E050E006
:102B8000040F151FA881B9810D931C93A5EDB0E02A
:102B90000D911D912D913C91AEE7B0E04D915D916D
:102BA0006D917C910E94C026A5EDB0E00D931D9320
:102BB0002D933D93A5EDB0E00D911D912D913C918C
:102BC000A1E7B0E04D915C91662777270E94C0266F
:102BD000A5EDB0E00D931D932D933D930E94161E1D
:102BE000A881B981AD90BC90ADEDB0E0AA0DBB1D40
:102BF0008C91AA81BB818D9388278D938D938C9323
:102C0000A881B9810E943225AA81BB810D911D91B5
:102C10002D913C9140E051E060E070E00E94492637
:102C2000AA81BB810D931D932D933D93AA81BB81F6
:102C30000D911D912D913C91A881B981AD90BC90D1
:102C4000ADEDB0E0AA0DBB1D4C9155276627772747
:102C50000E94C026AA81BB810D931D932D933D93A5
:102C6000009182000B3011F00C949616A881B98166
:102C70000E943225AA81BB810D911D912D913C911D
:102C800040E051E060E070E00E944926AA81BB81EB
:102C90000D931D932D933D93AA81BB810D911D91A1
:102CA0002D913C91A881B981AD90BC90ADEDB0E083
:102CB000AA0DBB1D4C915527662777270E94C02679
:102CC000AA81BB810D931D932D933D93A881B9815A
:102CD0000E943225AA81BB810D911D912D913C91BD
:102CE00040E051E060E070E00E944926AA81BB818B
:102CF0000D931D932D933D93AA81BB810D911D9141
:102D00002D913C91A881B981AD90BC90ADEDB0E022
:102D1000AA0DBB1D4C915527662777270E94C02618
:102D2000AA81BB810D931D932D933D93AA81BB81F5
:102D30000D911D912D913C91AE81BF810D931D93FD
:102D40002D933C9386E0481A8827580A24960895C4
:102D500080E0A881B9818C930027BB27A0E38C91E8
:102D600083FB0EF401E040E0041711F00C94BC1654
:102D700082E0A881B9818C930027BB27A0E38C91C6
:102D800084FB0EF401E040E0041711F00C94CC1623
:102D900081E0A881B9818C930027BB27A3E38C91A4
:102DA00081FB0EF401E040E0041711F00C94DC16F6
:102DB00083E0A881B9818C930027BB27A3E38C9182
:102DC00081FB0EF401E040E0041781E009F080E0AF
:102DD0008F930027BB27A0E38C9183FB0EF401E0C7
:102DE00040E0041781E009F080E09F918923882367
:102DF00011F40C94FF1684E0A881B9818C93089596
:102E000081E00E94392681E00E9439265398549827
:102E100080E081BB909A919AEF93FF93E0EFF1E00D
:102E20000E94FE25FF91EF9180E0AA81BB818C93E7
:102E300000917000003081E009F080E08F930091F4
:102E40007000023081E009F080E09F91892B882397
:102E500011F40C94D3170027BB27A0E38C9180FBBF
:102E60000EF401E040E0041711F00C943B1781E0F0
:102E7000AA81BB818C930027BB27A0E38C9181FBA7
:102E80000EF401E040E0041711F00C944C17AA81F5
:102E9000BB818C918E5F8C930027BB27A9E38C911B
:102EA00085FB0EF401E040E0041711F00C945D176F
:102EB000AA81BB818C918C5F8C930027BB27A9E3EF
:102EC0008C9184FB0EF401E040E0041711F00C94A7
:102ED0006E17AA81BB818C91885F8C93AA81BB817C
:102EE0000C91003018F011F00C9478170C94D11755
:102EF0008AE090E00E942A2680E0A881B9818C9324
:102F00000027BB27A0E38C9180FB0EF401E040E09A
:102F1000041711F00C94901781E0A881B9818C936B
:102F20000027BB27A0E38C9181FB0EF401E040E079
:102F3000041711F00C94A117A881B9818C918E5FB0
:102F40008C930027BB27A9E38C9185FB0EF401E04D
:102F500040E0041711F00C94B217A881B9818C914C
:102F60008C5F8C930027BB27A9E38C9184FB0EF424
:102F700001E040E0041711F00C94C317A881B98157
:102F80008C91885F8C93A881B9814C91AA81BB8177
:102F90000C91041711F40C94D11780E0AA81BB8125
:102FA0008C930C9479180027BB27A0E38C9180FBAD
:102FB0000EF401E041E0041711F00C94E31781E0F6
:102FC000AA81BB818C930027BB27A0E38C9181FB56
:102FD0000EF401E041E0041711F00C94F417AA81FB
:102FE000BB818C918E5F8C930027BB27A9E38C91CA
:102FF00085FB0EF401E041E0041711F00C94051874
:10300000AA81BB818C918C5F8C930027BB27A9E39D
:103010008C9184FB0EF401E041E0041711F00C9454
:103020001618AA81BB818C91885F8C93AA81BB8181
:103030000C91003018F011F00C9420180C947918B1
:103040008AE090E00E942A2680E0A881B9818C93D2
:103050000027BB27A0E38C9180FB0EF401E041E048
:10306000041711F00C94381881E0A881B9818C9371
:103070000027BB27A0E38C9181FB0EF401E041E027
:10308000041711F00C944918A881B9818C918E5FB6
:103090008C930027BB27A9E38C9185FB0EF401E0FC
:1030A00041E0041711F00C945A18A881B9818C9151
:1030B0008C5F8C930027BB27A9E38C9184FB0EF4D3
:1030C00001E041E0041711F00C946B18A881B9815C
:1030D0008C91885F8C93A881B9814C91AA81BB8126
:1030E0000C91041711F40C94791880E0AA81BB812B
:1030F0008C9300917000003081E009F080E08F93A4
:1031000000917000013081E009F080E09F91892BEF
:10311000882311F40C94CF18AA81BB810C91033041
:1031200011F00C94991882E0AA81BB818C930C94C5
:10313000CF18AA81BB810C91043081E008F480E0B3
:103140008F93AA81BB810C91073081E010F009F0C8
:1031500080E09F918923882311F40C94B51883E0B3
:10316000AA81BB818C930C94CF18AA81BB810C914E
:10317000083081E008F480E08F93AA81BB810C9134
:103180000F3081E010F009F080E09F9189238823BF
:1031900011F40C94CF1884E0AA81BB818C9381E058
:1031A00081BB9198539A549AAA81BB818C91AC812E
:1031B000BD818C9382E0481A8827580A2496089586
:1031C00081E00E94392681E00E943926AC81BD81D0
:1031D0008C91A881B9818C930E94060888EC90E0BC
:1031E0000E942A265A924A9281E0A42DB52D8C93F2
:1031F00081E00E9418250E948822229681E00E9488
:103200001425A895EBE6F0E0FA93EA930E94A8163D
:1032100022968AE090E00E942A2600916B000030FE
:1032200011F00C94011986E990E00E942A265A9226
:103230004A9280E0A42DB52D8C9381E00E94182540
:103240000E948822229681E00E94142584E690E064
:103250000E942A265A924A9280E0A42DB52D8C9382
:1032600081E00E9418250E948822229681E00E9417
:103270001425A895EBE6F0E0FA93EA930E94A816CD
:1032800022960E9408085A924A9281E0A42DB52DF8
:103290008C9381E00E9418250E948822229681E06A
:1032A0000E94142584E690E00E942A265A924A92AF
:1032B00080E0A42DB52D8C9381E00E9418250E94FA
:1032C0008822229681E00E9414258AE090E00E94E4
:1032D0002A265A924A9280E0A42DB52D8C9381E043
:1032E0000E9418250E948822229681E00E941425BF
:1032F0000E94060886E990E00E942A2600916B0051
:10330000003018F011F00C9487190C94391988E7E3
:1033100090E00E942A265A924A9281E0A42DB52D6F
:103320008C9381E00E9418250E949E1A229681E0CB
:103330000E941425A881B9810C91023011F00C94DF
:10334000E11900916B00013011F00C94AC1981E08F
:103350008093C5000C94DA19023011F00C94C41952
:1033600080E08093C5005A924A9281E0A42DB52D49
:103370008C9381E00E9418250E949E1A229681E07B
:103380000E9414250C94DA19033011F00C94DA1908
:1033900083E08093C5005A924A9282E0A42DB52D15
:1033A0008C9381E00E9418250E949E1A229681E04B
:1033B0000E941425EEE0F0E0A5ECB0E07BE70E946F
:1033C0005327A881B9810C91033011F00C940A1A8B
:1033D00000916B00013011F00C94F31981E080939F
:1033E00070000C94031A023011F00C94FC1980E068
:1033F000809370000C94031A033011F00C94031A9C
:1034000082E080937000E1E1F0E0A0E7B0E07BE7CC
:103410000E945327A881B9810C91013011F00C94BE
:103420005C1A00916B00013011F00C94231AA6EC89
:10343000B0E08C91897F8C93A6ECB0E08C91826097
:103440008C930C94551A023011F00C943D1AA6EC92
:10345000B0E08C91897F8C935A924A9281E0A42D9E
:10346000B52D8C9381E00E9418250E949E1A229609
:1034700081E00E9414250C94551A033011F00C942D
:10348000551AA6ECB0E08C9186608C935A924A92C1
:1034900084E0A42DB52D8C9381E00E9418250E9414
:1034A0009E1A229681E00E941425EFE0F0E0A6EC3F
:1034B000B0E07BE70E9453270E940A08A895EBE63C
:1034C000F0E0FA93EA930E94A816229685E090E035
:1034D0000E942A2600916B00003011F00C945E1AB5
:1034E00086E990E00E942A265A924A9280E0A42D12
:1034F000B52D8C9381E00E9418250E948822229687
:1035000081E00E94142586E990E00E942A265A92C2
:103510004A9280E0A42DB52D8C9381E00E9418255D
:103520000E948822229681E00E9414250E940808A9
:1035300082E0481A8827580A2496089581E00E945C
:10354000392681E0A881B9818C93AA81BB814C91F5
:10355000A881B9810C91041718F011F00C94CB1AC2
:103560005A924A9282E0A42DB52D8C9381E00E945C
:1035700018250E948822229681E00E9414258DE75A
:1035800090E00E942A26A881B9818C918F5F8C934C
:1035900010F40C94A51A81E0481A8827580A22963C
:1035A000089581E00E94392681E0A881B9818C9339
:1035B000A881B9810C91063018F011F00C94F41A1E
:1035C0000E9406088FE090E00E942A260E940808C8
:1035D00084E690E00E942A26A881B9818C918F5FB1
:1035E0008C9310F40C94D81A81E0481A8827580A52
:1035F000229608950E941626C39A88EC90E00E94B5
:103600002A2681B5886081BD0E944A215A924A9239
:1036100081E0A42DB52D8C9381E00E9418250E9495
:103620009621229681E00E94142581B5886181BD92
:10363000877F81BD84E690E00E942A26FF27E0E193
:10364000FA93EA935A924A928BE0A42DB52D8C936B
:1036500081E00E9418250E941E24249681E00E9489
:103660001425013051E0150711F00C944A1B5A92B1
:103670004A92A0ECB0E08D919C91A42DB52D8D9334
:103680009C9382E00E9418250E942E22229682E0BE
:103690000E9414255A924A9282E3A42DB52D8C9350
:1036A00081E00E9418250E949621229681E00E94C6
:1036B0001425C29AD89A82E390E00E942A2608959F
:1036C00081E00E94392681E00E9439268FEFAA818D
:1036D000BB818C9380E0A881B9818C93A881B9814A
:1036E0000C91073018F011F00C94831B91E0AA8123
:1036F000BB810E940C26A881B9818C918F5F8C932D
:1037000010F40C946E1B82E0481A8827580A2496FD
:10371000089581E00E94392681E00E94392681E0E7
:103720000E94392682E00E94392682E00E943926D2
:103730008FEFAA85BB858C9381E0A885B9858C9392
:10374000A885B9850C91003418F011F00C94B21BC7
:103750000E94601BA885B9858C918F5F8C9310F4B3
:103760000C94A01BC49881E0A885B9858C93A8858A
:10377000B9850C91003418F011F00C94C91B0E940B
:10378000601BA885B9858C918F5F8C9310F40C9485
:10379000B71B8AE090E00E942A26A895EE81FF815F
:1037A000FA93EA935A924A9280E4A42DB52D8C9311
:1037B00081E00E9418255A924A9200E010E020E031
:1037C00030E0A42DB52D0D931D932D933C9384E0F3
:1037D0000E9418250E94BF20269685E00E9414258D
:1037E000AE81BF810C91013011F40C94FA1BC49A84
:1037F0000C94101E81E0AA85BB858C93A89580E06F
:1038000090E0A881B9818D939C93EE81FF81FA931A
:10381000EA935A924A9281E4A42DB52D8C9381E0CB
:103820000E9418255A924A9200E010E020E030E011
:10383000A42DB52D0D931D932D933C9384E00E94F0
:1038400018250E94BF20269685E00E941425A88195
:10385000B9810E942B25AE81BF810C91003081E09F
:1038600009F080E08F93A881B9810D911C910030FF
:1038700050E0150781E009F080E09F91892B8823B3
:1038800011F40C94051CC49AA881B9810D911C9166
:10389000003050E0150711F00C94501C0C94101ED1
:1038A000A89584E690E00E942A26A895C49881E015
:1038B00090E00E942A26EE81FF81FA93EA935A92C1
:1038C0004A9280E5A42DB52D8C9381E00E941825A5
:1038D0005A924A9201E010E020E030E0A42DB52D8C
:1038E0000D931D932D933C9384E00E9418250E9414
:1038F000BF20269685E00E94142585E090E00E9476
:103900002A26C49A8AE090E00E942A26A89500E020
:1039100010E020E030E0AEE7B0E00D931D932D9372
:103920003C9300E010E020E030E0A5EDB0E00D9326
:103930001D932D933C930E94161E00E010E020E0A2
:1039400030E0A5EDB0E00D931D932D933C9300273F
:10395000ACE6B0E08C9180FB0EF401E041E004178E
:1039600011F00C94B51C0C94101EA8950091EA005F
:10397000023011F40C94491D8091A00280938200C2
:10398000A7EAB2E00D91112740E051E00E943F26E6
:10399000AA81BB810D931C93AA81BB810D911C91BF
:1039A000A6EAB2E04D915527040F151FAA81BB81ED
:1039B0000D931C93AA81BB810D911C912227332763
:1039C00040E050E061E070E00E944926AEE7B0E0E0
:1039D0000D931D932D933D93A5EAB2E00D91112710
:1039E00040E051E00E943F26AA81BB810D931C93C9
:1039F000AA81BB810D911C91A4EAB2E04D9155279B
:103A0000040F151FAA81BB810D931C93AEE7B0E094
:103A10000D911D912D913C91AA81BB814D915C919D
:103A2000662777270E94C026AEE7B0E00D931D936E
:103A30002D933D93009182000C3011F00C94231DC6
:103A40008BE080938200009182000E3011F00C9484
:103A50002C1D8BE080938200009182000F3011F0CA
:103A60000C94351D8BE080938200AEE7B0E00D91A1
:103A70001D912D913C91A5EDB0E00D931D932D93DB
:103A80003C930E94161EA5EDB0E00E9439250C94CF
:103A90005B1D00911401063411F00C94521D84E05A
:103AA0008093820000913001063411F00C945B1D6C
:103AB0008BE0809382008091EB00809373000091F3
:103AC0007300003011F00C94671D0C94101E0091CF
:103AD0007300003418F011F00C94701D0C94721DDA
:103AE0000C94101E8091EC00AE81BF818C9380916C
:103AF000ED00AC81BD818C93AC81BD819C91AE8188
:103B0000BF818C91A1E7B0E08D939C938091F400EC
:103B1000AE81BF818C938091F500AC81BD818C9387
:103B2000AC81BD819C91AE81BF818C91A4E7B0E056
:103B30008D939C93A4E7B0E00D911C91003050E070
:103B4000150711F00C94BA1D80910201AE81BF815E
:103B50008C9380910301AC81BD818C93AC81BD813C
:103B60009C91AE81BF818C91A4E7B0E08D939C9332
:103B70000C94BA1DA4E7B0E00D911C91003050E008
:103B8000150711F00C94C61D0C94101E02E010E0F5
:103B900020E030E0A4E7B0E04D915C916627772704
:103BA0000E944926A6E7B0E00D931D932D933D9307
:103BB000A6E7B0E00D911D912D913C91A1E7B0E0F9
:103BC0004D915C91662777270E94C026A6E7B0E05A
:103BD0000D931D932D933D93A6E7B0E00D911D919C
:103BE0002D913C91A5EDB0E04D915D916D917C9151
:103BF0000E94C026A6E7B0E00D931D932D933D9340
:103C0000A6E7B0E00D911D912D913C91A5EDB0E09E
:103C10000D931D932D933C9380E0AA85BB858C93D7
:103C200087E0481A8827580A2A96089581E00E945A
:103C3000392681E00E94392682E00E94392682E0FE
:103C40000E9439268FEFAE81BF818C9391E0AE81C7
:103C5000BF810E940C2691E0AE81BF810E940C269C
:103C600091E0AE81BF810E940C2691E0AE81BF81C0
:103C70000E940C2691E0AE81BF810E940C2691E04B
:103C8000AE81BF810E940C2691E0AE81BF810E946F
:103C90000C2691E0AE81BF810E940C2691E0AE819E
:103CA000BF810E940C2691E0AE81BF810E940C264C
:103CB00091E0AE81BF810E940C2691E0AE81BF8170
:103CC0000E940C2691E0AE81BF810E940C2691E0FB
:103CD000AE81BF810E940C2691E0AE81BF810E941F
:103CE0000C2691E0AE81BF810E940C26C49880E032
:103CF00090E0A881B9818D939C938FEF0E941D263F
:103D00000E941F260E941E26AE81BF818C93A8812F
:103D1000B9810E942B25AE81BF810C91003081E0DA
:103D200009F480E08F93A881B9810D911C91003036
:103D300050E0150781E009F080E09F91892B8823EE
:103D400011F40C947D1EA881B9810D911C91003055
:103D500050E0150711F00C94B41E80916C00816046
:103D600080936C000C94D91FEE81FF81FA93EA9343
:103D70005A924A9281E5A42DB52D8C9381E00E9440
:103D800018255A924A92A5EDB0E00D911D912D9102
:103D90003C91A42DB52D0D931D932D933C9384E060
:103DA0000E9418250E94BF20269685E00E941425B7
:103DB0000027ACE6B0E08C9180FB0EF401E041E01E
:103DC000041711F00C94E61E0C94D91FA895AE812F
:103DD000BF810C91003011F00C942B1F80E090E01B
:103DE000A881B9818D939C938FEF0E941D260E941C
:103DF0001F260E941E26AE81BF818C93A881B981A7
:103E00000E942B25AE81BF810C91003081E009F426
:103E100080E08F93A881B9810D911C91003050E012
:103E2000150781E009F080E09F91892B882311F428
:103E30000C94F41EA881B9810D911C91003050E0C2
:103E4000150711F00C942B1F80916C0081608093FA
:103E50006C000C94D91FAE81BF810C910F3F11F003
:103E60000C946F1F80E090E0A881B9818D939C93A2
:103E70008FEF0E941D260E941F260E941E26AE81E3
:103E8000BF818C93A881B9810E942B25AE81BF810F
:103E90000C910F3F81E009F480E08F93A881B981F4
:103EA0000D911C91003050E0150781E009F080E091
:103EB0009F91892B882311F40C94381FA881B98114
:103EC0000D911C91003050E0150711F00C946F1FFC
:103ED00080916C00816080936C000C94D91FAE813E
:103EE000BF810C910E3F11F40C947E1FC49A8091F7
:103EF0006C00816080936C000C94D91F80E090E08E
:103F0000AA81BB818D939C9380E0AE81BF818C930D
:103F1000AE81BF810C910F3F18F011F00C94C01FBF
:103F2000AA81BB810E942B258FEF0E941D260E9433
:103F30001F260E941E26AA81BB81AD90BC90ADEDCC
:103F4000B0E0AA0DBB1D8C93AA81BB810E942B25DA
:103F50008FEF0E941D260E941F260E941E26AA8106
:103F6000BB81AD90BC90ADEDB0E0AA0DBB1D8C93B4
:103F7000AE81BF818C918F5F8C9310F40C94881F5D
:103F80008FEF0E941D260E941F260E941E26AE81D2
:103F9000BF818C938FEF0E941D260E941F260E94D6
:103FA0001E26AE81BF818C93C49AA5EDB0E00E941D
:103FB0001C2586E0481A8827580A2896089582E02A
:103FC0000E94392681E00E94392680E0AE81BF81BF
:103FD0008C930E94601BC49880E090E0AA81BB8112
:103FE0008D939C938FEF0E941D260E941F260E9496
:103FF0001E26A881B9818C93AA81BB810E942B25A2
:10400000A881B9810C91003081E009F480E08F93A0
:10401000AA81BB810D911C91003050E0150781E011
:1040200009F080E09F91892B882311F40C94F21FF2
:10403000AA81BB810D911C91003050E0150711F051
:104040000C94292080916C00816080936C000C940A
:10405000B920E881F981FA93EA935A924A9281E56C
:10406000A42DB52D8C9381E00E9418255A924A9276
:10407000AA85BB850D911D912D913C91A42DB52D47
:104080000D931D932D933C9384E00E9418250E946C
:10409000BF20269685E00E941425A881B9810C9145
:1040A000003011F00C94802080E090E0AA81BB8168
:1040B0008D939C938FEF0E941D260E941F260E94C5
:1040C0001E26A881B9818C93AA81BB810E942B25D1
:1040D000A881B9810C91003081E009F480E08F93D0
:1040E000AA81BB810D911C91003050E0150781E041
:1040F00009F080E09F91892B882311F40C945A20B9
:10410000A881B9810C910F3F11F00C94B32080E08D
:1041100090E0AA81BB818D939C938FEF0E941D2616
:104120000E941F260E941E26A881B9818C93AA8115
:10413000BB810E942B25A881B9810C910F3F81E0A2
:1041400009F480E08F93AA81BB810D911C9100300E
:1041500050E0150781E009F080E09F91892B8823CA
:1041600011F40C948D20A881B9818C91AE81BF810E
:104170008C9383E0481A8827580A2496089584E08F
:104180000E94392681E00E94392682E00E94392669
:104190008FEFAA81BB818C9391E0AA81BB810E94A1
:1041A0000C2691E0A885B9850E940C26AE81BF81BE
:1041B0000D911D912D913C9140E052E060E070E046
:1041C0000E944926AC81BD810D931D932D933D9393
:1041D000AC81BD818F9314968E910E943F218E9168
:1041E0000E943F218E910E943F218E910E943F218B
:1041F00085E90E943F218F9180E090E0A881B981FC
:104200008D939C938FEF0E941D260E941F260E9473
:104210001E26AA81BB818C93A881B9810E942B257F
:10422000AA81BB810C910F3F81E009F480E08F935C
:10423000A881B9810D911C91003050E0150781E0F3
:1042400009F080E09F91892B882311F40C940221BE
:10425000A881B9810D911C91003050E0150711F033
:104260000C94372180916C00816080936C00AA814E
:10427000BB818C91AA85BB858C930C9444218FB90A
:10428000779BFECF8FB1089587E0481A8827580A98
:10429000269608955A924A9284E298E0A42DB52D6C
:1042A0008D939C9382E00E9418255A924A9280E056
:1042B000A42DB52D8C9381E00E9418250E94C32364
:1042C000249683E00E941425EF93FF93ECE8F1E03D
:1042D0000E94FE25FF91EF91BB27A0E38C9182FB0A
:1042E000DEF789E190E00E942A265A924A9280E203
:1042F00098E0A42DB52D8D939C9382E00E94182503
:104300005A924A9280E0A42DB52D8C9381E00E94B0
:1043100018250E94C323249683E00E94142589E176
:1043200090E00E942A260E944B22089582E00E947B
:10433000392600E011E0AA81BB814D9155270E94EA
:104340003F26A881B9810D931C93A881B9810D9155
:104350001C91AA81BB814D915527040F151FA8817F
:10436000B9810D931C935A924A92AA81BB818D9177
:104370009C91A42DB52D8D939C9382E00E941825CD
:104380005A924A928BE0A42DB52D8C9381E00E9425
:1043900018250E94C323249683E00E9414255A9274
:1043A0004A9280E298E0A42DB52D8D939C9382E0F3
:1043B0000E9418255A924A9280E0A42DB52D8C9324
:1043C00081E00E9418250E94C323249683E00E9466
:1043D000142582E0481A8827580A2296089582E018
:1043E0000E94392600E110E0AC81BD814D91552736
:1043F0000E943F26A881B9810D931C93A881B981A1
:104400000D911C91AA81BB814D915527040F151F59
:10441000A881B9810D931C935A924A92AA81BB81BB
:104420008D919C91A42DB52D8D939C9382E00E943B
:1044300018255A924A9282E0A42DB52D8C9381E0E2
:104440000E9418250E94C323249683E00E9414250D
:1044500082E0481A8827580A229608955A924A926A
:10446000AA81BB818D919C91A42DB52D8D939C9398
:1044700082E00E9418255A924A9283E0A42DB52D1D
:104480008C9381E00E9418250E94C323249683E028
:104490000E941425089581E00E94392681E00E943F
:1044A0003926C49AD898C29880E0A881B9818C93A3
:1044B00080E0AA81BB818C93AA81BB810C910F31D2
:1044C00018F011F00C94802291E0A881B9810E942B
:1044D0000C2691E0A881B9810E940C2691E0A88168
:1044E000B9810E940C2691E0A881B9810E940C2616
:1044F000AA81BB818C918F5F8C9310F40C945C2209
:10450000C29AD89A82E0481A8827580A24960895B1
:1045100081E00E9439265A924A9280E298E0A42DC6
:10452000B52D8D939C9382E00E9418255A924A9251
:1045300080E0A42DB52D8C9381E00E9418250E9467
:10454000C323249683E00E941425AA81BB810C9189
:10455000003011F00C94BB225A924A9280E0A42DB4
:10456000B52D8C9381E00E9418250E943523229658
:1045700081E00E941425AA81BB810C91013011F0C9
:104580000C94D1225A924A9285E6A42DB52D8C9393
:1045900081E00E9418250E943523229681E00E9426
:1045A0001425AA81BB810C91023011F00C94FE22DB
:1045B0005A924A9283E6A42DB52D8C9381E00E94F5
:1045C00018250E943523229681E00E94142588EC4C
:1045D00090E00E942A265A924A9280E0A42DB52D9E
:1045E0008C9381E00E9418250E943523229681E059
:1045F0000E94142582E390E00E942A26AA81BB81B2
:104600000C91033011F00C9427235A924A9282E6BF
:10461000A42DB52D8C9381E00E9418250E9435238E
:10462000229681E00E94142580E991E00E942A26CA
:104630005A924A9280E0A42DB52D8C9381E00E947D
:1046400018250E943523229681E00E9414258AE0D5
:1046500090E00E942A268AE090E00E942A2681E0CB
:10466000481A8827580A2296089581E00E94392620
:10467000C49AD898C298AA81BB810C91003018F0D6
:1046800011F00C9445230C947F2383E5A881B98114
:104690008C9391E0A881B9810E940C268FEEA881AD
:1046A000B9818C9391E0A881B9810E940C268EE695
:1046B000A881B9818C9391E0A881B9810E940C26D0
:1046C00091E0AA81BB810E940C2680E0A881B9817B
:1046D0008C9391E0A881B9810E940C2691E0A88179
:1046E000B9810E940C2691E0A881B9810E940C2614
:1046F00091E0A881B9810E940C260C94BB2385E42B
:10470000A881B9818C9391E0A881B9810E940C267F
:1047100088E7A881B9818C9391E0A881B9810E9432
:104720000C2689E6A881B9818C9391E0A881B98192
:104730000E940C2684E7A881B9818C9391E0A8811E
:10474000B9810E940C2680E0A881B9818C9391E008
:10475000A881B9810E940C2691E0A881B9810E94AC
:104760000C2691E0A881B9810E940C2691E0A881D5
:10477000B9810E940C26C29AD89A81E0481A8827EB
:10478000580A2296089581E00E943926C29AD89844
:104790005A924A9282E0A42DB52D8C9381E00E941A
:1047A00018250E947824229681E00E9414255A92AE
:1047B0004A92AC81BD818C91A42DB52D8C9381E062
:1047C0000E9418250E947824229681E00E941425D8
:1047D000AC81BD8111968C91A881B9818C935A923C
:1047E0004A92AA81BB818C91A42DB52D8C9381E036
:1047F0000E9418250E947824229681E00E941425A8
:10480000AC81BD818C91A881B9818C935A924A92D6
:10481000AA81BB818C91A42DB52D8C9381E00E943F
:1048200018250E947824229681E00E941425D89AA7
:1048300081E0481A8827580A2296089581E00E944C
:10484000392681E00E94392682E00E943926C29AE8
:10485000D8985A924A9283E0A42DB52D8C9381E08A
:104860000E9418250E947824229681E00E94142537
:104870005A924A92A885B9858C91A42DB52D8C9316
:1048800081E00E9418250E947824229681E00E94EF
:104890001425EC81FD81FA93EA930E947E242296EE
:1048A000EA81FB81FA93EA930E947E242296D89AA9
:1048B000AC81BD810D91112740E051E00E943F265F
:1048C000A881B9810D931C93A881B9810D911C9188
:1048D000AA81BB814D915527040F151FA885B98565
:1048E0000D931C9384E0481A8827580A2696089549
:1048F00091E0A881B9810E940C26089581E00E9470
:10490000392691E0A881B9810E940126A881B98148
:104910008C91AA81BB818C9381E0481A8827580A20
:104920002296089582E00E94392681E00E9439266D
:10493000C49ABB27A0E38C9182FBDEF7C298AC81BE
:10494000BD810D911C91003052E0150711F00C94BF
:10495000E12481E090E0AA81BB818D939C9380E06B
:10496000A881B9818C93A881B9810C910F3018F07E
:1049700011F00C94DF24BB27A0E38C9182FBDEF7BF
:1049800090E2AA81BB81AD90BC90ADEDB0E0AA0DE4
:10499000BB1D0E940C26AA81BB810D911C9140E297
:1049A00050E0040F151FAA81BB810D931C93A881B1
:1049B000B9818C918F5F8C9310F40C94B3240C9478
:1049C0000D2581E090E0AA81BB818D939C93AC8101
:1049D000BD814D915C91AA81BB810D911C91041701
:1049E000150718F011F00C940D25BB27A0E38C914E
:1049F00082FBDEF7C29A91E0AA81BB81AD90BC90A8
:104A0000ADEDB0E0AA0DBB1D0E940C26AA81BB81B2
:104A10000E942B2510F40C94E724C29A83E0481AD4
:104A20008827580A24960895481A8827580A08950E
:104A3000480E8827581E08950D911D912D913C9187
:104A400081E0080F8827181F281F381F3C932E93DA
:104A50001E930E930895ED91FC91EF5FFF4FFC9331
:104A6000EE930895ED91FC91E150F040FC93EE93AC
:104A700008950D911D912D913C91015010402040C1
:104A800030403C932E931E930E9308954091DF0285
:104A90005091E0020DE815E30E945A2549E156E3E2
:104AA000040F151F0093DF021093E0024981588123
:104AB0000C94802509D00E943F2600FC10D0089558
:104AC00003D01ED001F8F9CF0024E89457FF02C0AC
:104AD00009D0689400F80BD010F80124089502D092
:104AE00009D00895509540954F5F5F4F0895E89421
:104AF00017FF0895009510950F5F1F4F6894089554
:104B0000352F242FE894452B11F468940895512FE4
:104B1000402F0027112780E1440F551F001F111F50
:104B2000021B130B416018F4020F131F4E7F8A956E
:104B300099F708958F938D918823E9F711978F91B5
:104B4000089588EE93E086D03197D9F7089500FC58
:104B500005D0089530D005D001F8F9CF37D03FD037
:104B60000895842F952FA62FB72FE894452B462B19
:104B7000472B11F468940895402F512F622F732F03
:104B80000027112722273327F0E2440F551F661F05
:104B9000771F001F111F221F331F081B190B2A0B21
:104BA0003B0B416028F4080F191F2A1F3B1F4E7F43
:104BB000FA9559F708950024E89477FF02C006D0CB
:104BC000689400F809D010F80124089512D04F5FBE
:104BD0005F4F6F4F7F4F0895E89437FF089500951A
:104BE0001095209530950F5F1F4F2F4F3F4F6894C2
:104BF0000895409550956095709508953197F1F717
:104C000008950E941D268C910E941F268D939A95CF
:104C1000D1F70E941E2608950E941D268D910E94A4
:104C20001F269A95D9F70E941E260895BF9ABE980E
:104C3000C69ABD9A80E58DB90895089508958FB9F3
:104C4000779BFECF8FB10895689462F80895E89439
:104C500062F80895EF93FF93EE27E82BE92B31F0EC
:104C6000E0EDF7E03197F1F70197D1F7FF91EF9180
:104C700008955A924A92480E8827581E08950F9216
:104C8000B801469F8001479F100D569F100D0F9051
:104C900008950F921F922F92C801D901489F800159
:104CA0004A9F90014B9F202C499F100D211D321DC2
:104CB0005A9F202C589F100D211D321D599F200DE9
:104CC000311D689F200D311D699F300D789F300D7B
:104CD0002F901F900F9008950E9472260D92002031
:104CE000D9F70895C895319600200895819104D090
:104CF0008D938823D9F70895813618F08B3708F4FF
:104D00008F7D08952E2E3F2E992781918D3209F0A7
:104D100093958823D1F79A95E22DF32D112361F015
:104D2000091718F011F0101B01C0191B28F021F011
:104D300080E28D931A95E9F780818D3219F48D9375
:104D4000319604C0222311F08BE28D93091738F0BD
:104D500031F0091B21F080E38D930A95E9F78191E9
:104D60008D938823E1F7332351F0EA2FFB2F3196FF
:104D700033958E9182933A95E1F78EE28C93089564
:104D8000040F151F261F371F0895041B150B260B34
:104D9000370B089504171507260737070895000FE6
:104DA000111F221F331F08950095109520953095EF
:104DB0000F5F1F4F2F4F3F4F0895019110810EC07D
:104DC00001911191219130810BC00191108117FF48
:104DD00005C03FEF2FEF04C00081112722273327A2
:104DE00037FF03C0E1DF8DE28D93CF93DF93CF9246
:104DF000DF92EF92AA24BB24CC24DD24EE2440E2EF
:104E0000CAE0DD2755E093E38881890F87FD9F7015
:104E100083FD907F891B89935A95A9F7C0DFAA1C4F
:104E2000BB1CCC1CDD1CEE1C4A9551F7E894EFE04E
:104E3000FF2782910ED0EB30E0F71EF068948A2DA8
:104E40000CD088278D93EF90DF90CF90DF91CF919A
:104E50000895982F829501D0892F8F70805D26F05C
:104E6000803309F4089568948D93089588278D936D
:104E7000089581918D938823E1F708950991919187
:104E8000992351F08A95D9F7319781918D930A959D
:104E900019F08823D1F70895E9CFE199FECFEEBB51
:104EA000FFBB3196089591E001C092E07B3751F449
:104EB0007FB7F894F2DF8D918DBBE29AE19A9A95D3
:104EC000C9F77FBF7727089591E001C092E0E5DF41
:104ED000E09A8DB38D939A95D1F70895FF93881B2F
:104EE000F9E0001FFA9511F4FF910895881F841BC3
:104EF00018F4840F8894F5CF0894F3CF689401C018
:104F0000E894AF93BF938D9116F0919103C00E94E6
:104F10007226902D891718F011F48823A1F7BF91FC
:104F2000AF9108954F005A00590048004200434F86
:084F30004E46494700002E0027
:00000001FF
